:1000000019C032C031C030C02FC02EC02DC02CC08E
:100010002BC02AC029C028C027C026C025C024C0A4
:1000200023C022C021C020C01FC01EC01DC01CC0D4
:100030001BC01AC011241FBECFEFD2E0DEBFCDBF60
:1000400011E0A0E0B1E0EAEBF0E002C005900D9213
:10005000A030B107D9F711E0A0E0B1E001C01D92D6
:10006000A030B107E1F710C0CBCF181619065CF429
:1000700028EE33E02250304012161306DCF30197CD
:1000800018161906ACF30895CFEFD2E0DEBFCDBF4E
:100090008FEB85B980EC84B91BB88FEF8AB981E00A
:1000A00088B917B8C82F8C2F992787FD9095CF5FF7
:0A00B000DCDF8BB180958BB9F6CF31
:00000001FF
